:100000000C944C000C9469000C9469000C946900E9
:100010000C9469000C9469000C9469000C946900BC
:100020000C9469000C9469000C9469000C947A019A
:100030000C9469000C9469000C9469000C9469009C
:100040000C9469000C9469000C94D6000C9469001F
:100050000C9469000C946B000C9469000C9469007A
:100060000C9469000C9469000D0A002C0024475080
:10007000524D4300244750474741002E6C6F6700A4
:10008000244750524D430024505352463130362CB1
:1000900032312A30460D0A0011241FBECFEFD4E0C2
:1000A000DEBFCDBF11E0A0E0B1E0ECEEF2E202C0B5
:1000B00005900D92A630B107D9F714E0A6E0B1E0A3
:1000C00001C01D92A734B107E1F70E94BA010C9458
:1000D00075110C9400001F920F920FB60F9211240D
:1000E0002F933F938F9320917800309179008091E6
:1000F0007C00203D310570F4809109018F3030F093
:100100008091690181608093690106C08F5F80934F
:10011000090102C01092090181E02C32380770F009
:10012000809108018F3030F0809169018E7F80933B
:10013000690106C08F5F8093080102C01092080118
:1001400030936F0120936E0182E480937C00809154
:100150007C0030930A022093090281E480937C00A2
:100160008FED80937A008F913F912F910F900FBE6A
:100170000F901F90189560E070E081EA96E3089573
:10018000F894E1ECF0E0108210927101109270018D
:100190001092720181E48093C40088E98083809189
:1001A00069018D7F80936901789408951F920F9261
:1001B0000FB60F9211248F939F93EF93FF9390911B
:1001C000C60080917201863988F48F5F8093720136
:1001D00080917001E82FFF27E059FE4F93838F5FD6
:1001E000863908F080E08093700105C08091690134
:1001F000826080936901FF91EF919F918F910F90A1
:100200000FBE0F901F90189590E08091690180FFBC
:1002100003C080E090E00895209171018091720107
:10022000882319F420E030E015C0E22FFF27E059C1
:10023000FE4F3381E22FEF5FF8948091720181507D
:10024000809372017894E63908F0E0E0E093710160
:10025000232F33278091690181FF03C00E94C000D2
:10026000D3CF822F222389F2992311F4243269F605
:10027000E92FFF27E95EFE4F20839F5F8A3021F040
:10028000923508F0C1CFC1CF892F99270895982FB3
:100290000FC083E085BD90931601809116018823DD
:1002A000E1F715BC90931601809116018823E1F7C0
:1002B000615078F70895DC01FB016F5F7F4F9491E7
:1002C000992329F08C91981711F41196F5CF892F65
:1002D00099270895FC010AC08081813218F480E0DA
:1002E00090E0089531968C32B9F761506623A1F7FA
:1002F000CF0108951F920F920FB60F9211242F93E2
:100300003F934F935F936F937F938F939F93AF939D
:10031000BF93EF93FF9380911601882319F08150CA
:1003200080931601809106019091070101969093A8
:100330000701809306018055964448F0109207010A
:1003400010920601809169018460809369010E9486
:10035000C80DFF91EF91BF91AF919F918F917F91C8
:100360006F915F914F913F912F910F900FBE0F9022
:100370001F901895CDEFD4E0DEBFCDBF8DE085B9DD
:100380008EE284B98FE388B917B88EEA8BB982E51B
:100390008AB980E58CBD81E08DBD83ED90E39093BB
:1003A0008900809388008AE08093810082E08093B6
:1003B0006F0082E187BD82E484BD81E480937C008C
:1003C0008FED80937A00789467E272E080E00E947B
:1003D000EF08CC24DD2447E1E42E41E0F42E3BE09D
:1003E000A32E32E0B32E2E010894411C511C22E1B1
:1003F000622E21E0722E9AE6892E91E0992E89E0F4
:10040000282E312C2E0C3F1C1092C100299884E616
:10041000809316018091690180FF03C084E6809378
:100420001601809116018823A9F7299A8FEF8093EE
:1004300016018091690180FD05C080E00E94BF0D1A
:1004400081FF03C08FEF80931601809116018823EE
:1004500081F761E085E00E9447010E94C00027E823
:1004600030E006C08091C00085FFFCCF9093C600AD
:10047000F9012F5F3F4F94919923A1F70E94040146
:10048000882309F4C1CF60E870E0C7010E945B01D6
:10049000882329F462E0C7010E946A016C01C1143B
:1004A000D10461F3F6018081813441F769E0C7012D
:1004B0000E946A016C01009711F463E0A8C0FC017E
:1004C0008481958190931801809317018281938193
:1004D00090931A01809319018081918190931C015E
:1004E00080931B016BE770E08DE191E00E948D101D
:1004F00042E1B701C5010E944409892B09F086C079
:1005000040911502509116026091170270911802E5
:10051000C5010E948B05892B09F078C062E085E057
:100520000E94470165C064E770E0C7010E945B015B
:10053000882341F06DE670E0C7010E945B018823CB
:1005400009F044C0012F11279201A801B701C5018C
:100550000E94C006892B09F052C089819A81081730
:10056000190709F04CC04AE050E0B30180916E01D8
:1005700090916F010E94B8104AE050E0B401809160
:10058000090290910A020E94B810B301C7010E94AB
:10059000B1106BE670E08BE191E00E948D10B40128
:1005A0008CE191E00E94B11068E670E0C1010E9408
:1005B0008D1092014BE050E0B701C5010E94C006CA
:1005C000892BE9F489819A810B97C9F4809169019B
:1005D00082FF0EC0C5010E945D06892B11F066E006
:1005E00016C0F894809169018B7F8093690178949B
:1005F0000E940401182F882309F095CF0FC065E0F1
:1006000006C061E082E30E944701FECE64E01092E2
:10061000C100299889E10E944701FFCF1092C100D3
:100620002998C5010E94B406892B59F367E0EFCFE2
:10063000CF93DF93C0910A01D0910B01BC016250AE
:1006400070408E899F8902976817790728F020E00B
:1006500030E040E050E012C0882799272D8D3327E5
:10066000442755270E94E9109B01AC01888999898C
:10067000AA89BB89280F391F4A1F5B1FCA01B9010C
:10068000DF91CF910895FC01892B61F080819181E8
:100690008617970739F480E00E94BF0D9927817073
:1006A000907008958CE090E00895A0E0B0E0EBE554
:1006B000F3E00C942E114B015C01C0910A01D09122
:1006C0000B01CC80DD80EE80FF80C616D706E806E1
:1006D000F90609F44FC08F8D8823A1F180E2682EBE
:1006E000712C6C0E7D1E01E0A7019601B30180E024
:1006F0000E94D30E892BD9F51F8E8C899D89AA273C
:10070000BB27288539854A855B85820F931FA41FE7
:10071000B51FC816D906EA06FB06A0F41E8D10C048
:100720008C899D89AA27BB27C80ED91EEA1EFB1EED
:1007300001E0A7019601B30180E00E94D30E1150A1
:10074000123070F781149104A104B10499F0BE0134
:10075000605E7F4F01E0A501940180E00E94510F8F
:10076000892B29F48C829D82AE82BF8203C080E0F7
:1007700090E002C081E090E0EEE0CDB7DEB70C94EF
:100780004A11A0E0B0E0E7ECF3E00C942D11EC018D
:100790005B0180900A0190900B01F401C084D18428
:1007A000E284F384848D813021F0823009F070C0BE
:1007B00056C08E01000F111F0C0F1D1F16950795B7
:1007C000B801672F77276695882799276C0D7D1DBF
:1007D0008E1D9F1D0E945503882309F459C060E2B5
:1007E000662E712C680C791CF801F170E60DF71D6E
:1007F000CE0181709070582E882339F080818F70DF
:100800009A2D9295907F982B01C09A2D9083E801A4
:10081000219681E0F401878FBE01672F77276695C7
:10082000882799276C0D7D1D8E1D9F1D0E945503E5
:10083000882371F1FE01F170E60DF71D552039F0A6
:1008400044E0B694A7944A95E1F72A2D06C020818A
:10085000207F8B2D99278F70282B208313C06D2F1D
:100860007727882799276C0D7D1D8E1D9F1D0E945F
:100870005503882369F0CC0FDD1FD170C80DD91D39
:10088000B9A2A8A281E0F401878F81E090E002C0C4
:1008900080E090E0EFE0CDB7DEB70C944911A0E026
:1008A000B0E0E5E5F4E00C9431118C01E0900A0130
:1008B000F0900B01029708F467C0F70186899789C9
:1008C0000817190708F060C0A084B184C284D384DB
:1008D000848D813021F0823009F056C040C0E8019B
:1008E000CC0FDD1FC00FD11FD695C795BE01672F56
:1008F00077276695882799276A0D7B1D8C1D9D1D7E
:100900000E945503882309F43FC0FE01F170EE0DEB
:10091000FF1D90A02196BE01672F77276695882737
:1009200099276A0D7B1D8C1D9D1D0E9455038823F0
:1009300059F1292D3327D170EC0EFD1EF70180A14E
:100940009927982F8827822B932B00FF06C024E03D
:10095000969587952A95E1F719C09F7017C0612F6A
:100960007727882799276A0D7B1D8C1D9D1D0E9466
:100970005503882349F0000F111F1170E00EF11E7E
:10098000F70180A191A102C081E090E0EBE0CDB73A
:10099000DEB70C944D11EF92FF920F931F93CF93FC
:1009A000DF93EC01E0900A01F0900B010A811B81BA
:1009B0000F5F1F4FC8018F709070892BD1F58A850A
:1009C0009B85AC85BD850196A11DB11D8A879B873E
:1009D000AC87BD87488559854115510539F4F70124
:1009E000828193810817190720F128C0F701858DAE
:1009F000992701979801B4E036952795BA95E1F7C4
:100A000082239323892BA9F4CA010E944F049C01DD
:100A10000297A0F0F701868997892817390770F4A3
:100A200039872887C9010E9418036A877B878C87CA
:100A30009D871B830A8381E090E002C080E090E004
:100A4000E6E0CDB7DEB70C945211A0E0B0E0EBE2E7
:100A5000F5E00C9432117C01A0900A01B0900B01DA
:100A6000F501C688D788009749F4008D118D0230B2
:100A7000110580F00C151D0568F40EC00E944F048E
:100A800082309105E8F18C159D0510F4BC013DC044
:100A9000870102C001E010E0E8012196CC15DD05D8
:100AA00028F00230110578F1C2E0D0E0CE010E94BA
:100AB0004F04009731F0019719F1C017D10719F1D0
:100AC000ECCF6FEF7FEFCE010E94C1038823C1F00E
:100AD000E114F10431F0BE01C7010E94C103882373
:100AE00079F0F501D18FC08F828D938DFFEF8F3F0D
:100AF0009F0721F00197F501938F828FBE0105C0FA
:100B000061E070E002C060E070E0CB01EAE0CDB7E8
:100B1000DEB70C944E11A0E0B0E0E1E9F5E00C94F2
:100B20002A11EC013A014B014C805D80688179818A
:100B3000C2010E9443031C01892B09F0B8C02A811D
:100B400022230CF4B1C08A859B85AC85BD858615B2
:100B50009705A805B90520F421FD02C03C014D010F
:100B60001E821F821886198681E08B8361147104AE
:100B70008104910409F47EC02E853F85211531053D
:100B800071F480E090E00E9425059C018130910580
:100B900009F487C09F878E87892B09F46BC0F20107
:100BA000858DE82EFF240027112789E0EE0CFF1C1D
:100BB000001F111F8A95D1F7398B288BE614F70493
:100BC0000805190550F58A8181FF04C0C9010E94FA
:100BD000250503C0C9010E944F049C010097D9F06C
:100BE000019709F45EC0F2018689978928173907B1
:100BF00008F057C08E819F81A885B9858E0D9F1DF5
:100C0000A01FB11F8E839F83A887B9876E187F08A6
:100C1000800A910AD1CF3701480164015301089439
:100C2000A108B108C108D10809E0D694C794B794C7
:100C3000A7940A95D1F7EA2CFF2400271127C901B0
:100C40000E941803E60EF71E081F191FEA8AFB8A86
:100C50000C8B1D8BF201858D8A198B838E819F8170
:100C6000A885B985860D971DA81DB91D8E839F8304
:100C7000A887B9876A8161FF1AC02E813F814885A4
:100C800059858A859B85AC85BD8582179307A40706
:100C9000B50768F42A873B874C875D8760626A8363
:100CA00006C08A8180688A8318E0212E312CC10118
:100CB000E2E1CDB7DEB70C944611EF92FF920F93AD
:100CC0001F93CF93DF93EC01688179818C819D81A3
:100CD0000E9443037C01892B09F040C08A8185FF73
:100CE0003DC06E897F89888D998D0E945503882328
:100CF00091F10A8D1B8DF8018385806283878A8537
:100D00009B85AC85BD85848F958FA68FB78F8E858B
:100D10009F85938F828F0E94BB00F801668B778B33
:100D2000808F918F8A818F7D8A83E0910A01F09173
:100D30000B0181E0878F60E070E080E090E00E942E
:100D40005503882341F040E050E063E080E00E94DA
:100D5000E80D892B19F098E0E92EF12CC701E6E0A7
:100D6000CDB7DEB70C945211CF93DF93EC010E9404
:100D70005D06009711F41D821C82DF91CF910895CA
:100D8000A0E0B0E0E6ECF6E00C942C11EC018B0155
:100D90007A013901CC80DD80F901118210826881ED
:100DA0007981C6010E9443034C01892B09F01AC1C5
:100DB0008A8188230CF413C181FD04C0E6E08E2EE5
:100DC000912C10C12A853B854C855D85C701AA27DA
:100DD000BB27820F931FA41FB51F82179307A40779
:100DE000B50708F4FFC0580170E2472E512C4C0C97
:100DF0005D1CD9C02E813F8148855985DA01C90122
:100E00009170A070B0700097A105B10509F093C072
:100E10008B8181508B83882349F02A893B894C89B7
:100E20005D892F5F3F4F4F4F5F4F30C02115310518
:100E30004105510569F42E853F852115310589F459
:100E400080E090E00E9425059C019F878E8705C069
:100E5000888999890E9425059C012115310509F48D
:100E6000A6C02130310509F4B7C0F60186899789FB
:100E70002817390708F0B0C0398B288BC9010E94A8
:100E800018039B01AC01F601858D8B832A8B3B8B6C
:100E90004C8B5D8B8701012F11270695002361F193
:100EA0008B81102F801708F4182F012FB50180E0D7
:100EB0000E94D30E892B09F08FC08B818F5F811B1D
:100EC0008B83812F992701979C01442737FD4095FB
:100ED000542F8C010F5F1F4F8A899B89AC89BD8974
:100EE000820F931FA41FB51F8A8B9B8BAC8BBD8B6E
:100EF000102F0027110F3DC02E813F814885598555
:100F00008A859B85AC85BD85281739074A075B070D
:100F100090F060E070E080E090E00E94550388234C
:100F200009F45AC08A899B89AC89BD89F6018483FA
:100F30009583A683B7836A897B898C899D890E9462
:100F40005503882309F448C08E819F81917020E069
:100F500032E0281B390B87012E153F0508F4890163
:100F6000A801B501840D951D0E94A11081E0F60134
:100F7000878FA00EB11EC801AA27BB272E813F81F3
:100F800048855985280F391F4A1F5B1F2E833F83D1
:100F900048875987F30180819181800F911F918348
:100FA0008083E01AF10AE114F10409F023CF2E81C5
:100FB0003F81488559858A859B85AC85BD8582178B
:100FC0009307A407B50720F42A873B874C875D87E2
:100FD0008A8180628A8306C08A8180688A8328E049
:100FE000822E912CC401E0E1CDB7DEB70C944811FC
:100FF000A0E0B0E0EEEFF7E00C942C11EC018B01D7
:101000007A0139018C809D80F901118210826881FA
:101010007981C4010E9443035C01892B09F0D9C086
:101020008A8188230CF4D2C080FD04C006E0A02E83
:10103000B12CCFC02A853B854C855D858E819F81F3
:10104000A885B985281B390B4A0B5B0BC701AA275A
:10105000BB27281739074A075B0708F4790168019D
:1010600010E2412E512C480C591CA8C02E813F8102
:1010700048855985DA01C9019170A070B070009758
:10108000A105B10509F066C08B8181508B8388234F
:1010900049F02A893B894C895D892F5F3F4F4F4F2B
:1010A0005F4F22C0211531054105510519F42E85E8
:1010B0003F8505C0888999890E944F049C01223090
:1010C000310508F480C0F40186899789281739070B
:1010D00008F079C0398B288BC9010E9418039B0145
:1010E000AC01F401858D8B832A8B3B8B4C8B5D8B04
:1010F0008701012F11270695002361F18B81102FA5
:10110000801708F4182F012FB60180E00E94510FBC
:10111000892B09F058C08B818F5F811B8B83812FB6
:10112000992701979C01442737FD4095542F8C0146
:101130000F5F1F4F8A899B89AC89BD89820F931FDE
:10114000A41FB51F8A8B9B8BAC8BBD8B102F0027E8
:10115000110F1AC06A897B898C899D890E94550369
:10116000882389F16E817F81717080E092E0861B17
:10117000970B87018E159F0508F48C01640D751D72
:10118000A801C6010E94A110C00ED11EC801AA2745
:10119000BB272E813F8148855985280F391F4A1F5B
:1011A0005B1F2E833F8348875987F301808191819C
:1011B000800F911F91838083E01AF10AE114F104FA
:1011C00009F054CF06C08A8180688A83F8E0AF2E88
:1011D000B12CC501E0E1CDB7DEB70C944811FB019D
:1011E000882319F085E090E00895A0910A01B0915C
:1011F0000B0170930B0160930A01109729F080E2B4
:1012000092E01D920197E9F7309719F480E090E0A1
:10121000089580E292E011920197E9F780E090E072
:1012200008950F93CF93DF939B01AC01C0910A0106
:10123000D0910B01BE01605E7F4F01E080E00E9413
:10124000510F892BD9F4C25EDD4F88819981CE512F
:10125000D24085559A4A91F400E043E050E060E0C6
:1012600071E0CE018A5A9F4F0E949410892B09F495
:1012700001E081E00827802F992702C082E090E0FA
:10128000DF91CF910F910895ADE1B0E0EAE4F9E08C
:101290000C942A119D8F8C8F6B01A0900A01B09045
:1012A0000B01FC0115821482F42FFF71FB8F03C028
:1012B0000894C11CD11CD6018C918032C9F38F32A5
:1012C00019F40894C11CD11CA114B10409F415C16E
:1012D0001B8D1E71F501848D882361F080E00E94D2
:1012E000BF0D992780FD06C0112309F429C382FD93
:1012F00007C126C380E292E0D5011D920197E9F76C
:1013000080E00E94AE0F992780FF03C021E030E00B
:1013100045C3112311F082FDF3C060E070E080E06E
:1013200090E00E941109813021F0EE24FF24870112
:101330001EC0E2EEF1E0AE0EBF1ED5018C91EEE1D3
:10134000FEEFAE0EBF1E882309F4DDC026EE31E0AD
:10135000A20EB31ED501ED90FD900D911C91EAE116
:10136000FEEFAE0EBF1EC801B7010E94110988230F
:1013700009F0C9C0F50183A594A58050924009F0F9
:10138000C2C0F50166A977A96115710519F0882712
:1013900099270DC024E430E0A20EB31ED5016D9153
:1013A0007D918D919C91ECEBFFEFAE0EBF1EF50190
:1013B000758B648B20A9268F3327442755270E94DD
:1013C000E9103B014C01A501425D5F4FF50186A587
:1013D00097A5AA27BB27E80EF91E0A1F1B1FE08648
:1013E000F1860287138785A5858F21A932A93383CA
:1013F000228363A974A96115710521F07B0100277F
:1014000011270DC080E490E0A80EB91ED501ED9023
:10141000FD900D911C91E0ECFFEFAE0EBF1EDA01C6
:101420008D919C91AA27BB27E81AF90A0A0B1B0B7E
:10143000E618F70808091909E4E036952795EA95B2
:10144000E1F7C901AA27BB27E81AF90A0A0B1B0B07
:10145000F501258D332744275527C801B7010E9480
:1014600008112E5F3F4F4F4F5F4FF501378B268B93
:10147000283FFFE03F07F0E04F07F0E05F0710F480
:1014800061E006C0285F3F4F40405040E0F562E019
:10149000F5012085318542855385D401C301820F32
:1014A000931FA41FB51F84879587A687B78782815E
:1014B000938174E0969587957A95E1F7AA27BB27E3
:1014C000820F931FA41FB51F860D971DA81DB91D60
:1014D000808B918BA28BB38B648F8FEF9FEF938F59
:1014E000828F80910C0190910D01019690930D01D6
:1014F00080930C019183808323C22AE030E04EC2A6
:1015000029E030E04BC22BE030E048C236014E010A
:101510000894811C911C50E2452E512C4E0E5F1EEA
:101520004DE0242E312C2C0E3D1E4BE050E060E2AD
:1015300070E0C4010E94AA1040E068E030E058E189
:1015400002C048E06BE0D3012D913D01222311F050
:101550002F3251F4442309F443C053235C87822F74
:10156000992787FD90953EC0922F2132C8F12F37E1
:10157000B9F12E3239F430FD33C0442389F14930BA
:1015800000F32EC0223261F12A3208F12D3240F1EF
:101590002A33E8F0203420F130FD19C02C3701F156
:1015A000822F8B558330E0F0865E8A3128F46830D4
:1015B00011F4577F01C05F7E822F81568A3138F443
:1015C000922F9052683011F4386001C03061461794
:1015D00038F43E7FF401E40FF11D90834F5FB3CFE9
:1015E00081E090E0D82EB1E08B1719F424E030E0D0
:1015F00055C06F89788D898D9A8D0E9455038823F7
:1016000019F428E030E04AC00F8518890F70107077
:1016100035E0000F111F3A95E1F7040D151DF80193
:1016200080818823A9F0853E71F0F8018385E82E3A
:10163000FF24E3FC08C04BE050E0B401C8010E9465
:101640009410892B51F0C1010E94CB04882389F6A4
:10165000DD2059F422E030E021C0DD2021F46801D2
:1016600020E030E01BC0E4FC03C023E030E016C003
:10167000F801828D938D9C8B8B8B9E8B8D8B0E9422
:1016800018036F8B788F898F9A8F82E090E0988B08
:101690008F874BCF20E030E0CC24DD24FB8D4F2F13
:1016A0005527CA018C719070892B09F4FEC0211551
:1016B000310509F48FC02230310509F06FC1609007
:1016C0000A0170900B010B891C890115110551F05D
:1016D0001E8B0D8BC8010E9418036F8B788F898F2A
:1016E0009A8F09C0F30184859585A685B7858F8B70
:1016F000988FA98FBA8F188A1F8620E2E22EF12CCC
:10170000E60CF71C9DE0492E512C4C0E5D1E6F8996
:10171000788D898D9A8D0E945503882309F40AC11A
:101720004701CF84D888FFE0CF22DD2485E0CC0CB0
:10173000DD1C8A95E1F7CE0CDF1CD6018C91882345
:1017400009F418C1853E09F415C1C2010E94CB04F9
:101750008823E9F6012B09F4EAC08D899E890E944D
:1017600025058C01009709F4E2C0019709F4E2C055
:1017700060E070E080E090E00E945503882309F467
:10178000D9C0C8010E9418036B017C01F301648376
:1017900075838683978380E092E0D4011D92019740
:1017A000E9F7158D10C001E0A7019601B40180E0B2
:1017B0000E94D30E892B09F0BDC00894C11CD11C16
:1017C000E11CF11C1150112371F781E0F301878FA7
:1017D0006401D0C042FF03C027E030E0DFC0C11485
:1017E000D10409F4A4C0F6018385817109F09FC07A
:1017F00043FF46C0828C938C138E128E148E158EEE
:10180000168E178E81E0F501878F24803580468003
:101810005780E0900A01F0900B0184011BC0C801C1
:101820000E944F043C01019709F484C060E070E01D
:10183000C8010E94C103882309F47CC0F701828D8E
:10184000938DFFEF8F3F9F0721F00196F701938F54
:10185000828F83010230110530F0F7018689978964
:1018600008171907E0F2C201B1010E94550388234D
:1018700009F460C0089481089108F501918E808E6A
:10188000FB8DF3FF23C080E2F60183870E94BB003B
:10189000F601668B778B808F918F66877787808B39
:1018A000918B81E0F501878F11C02115310509F079
:1018B00075C0C114D10409F440C0F601838599278D
:1018C00084FD3BC041FF02C080FD31C0F501848131
:1018D0009581A681B781EC8DFD8D868B978BA08F2E
:1018E000B18FD38EC28E2B8D2283F601828D938D84
:1018F000EC8DFD8D97878687F601848D958DA68D5D
:10190000B78DEC8DFD8D82879387A487B58716826E
:1019100017821086118681E08383B582A482D50167
:101920008D919C919183808320E030E037C026E048
:1019300030E034C028E030E031C022E030E02EC09A
:10194000E0910A01F0910B01848595851C8A1B8A20
:101950001E8A1D8AAA27BB278F8B988FA98FBA8FC3
:10196000188A1F86FA8BE98BD6018C91882309F49B
:1019700091CECCCD80E2F60111928A95E9F7F6017D
:10198000DE0111968BE00D9001928150E1F78C857C
:10199000F6018487FB8DF860FB8F72CFC901E2E10D
:1019A0006D960C94461182E3809310018FEF8EBDEB
:1019B0000DB407FEFDCF8EB58FEF8EBD0DB407FEC3
:1019C000FDCF8EB5282F33278F3F21F08091100156
:1019D000882391F7C9010895FC018AE080930F01E3
:1019E0008FEF8EBD0DB407FEFDCF8EB58F3F29F46E
:1019F00080910F01882329F1F3CF8E3F11F58FEFEE
:101A00008EBD0DB407FEFDCF8EB580838FEF8EBDEA
:101A10000DB407FEFDCF8EB581836250704011F08A
:101A20003296EDCF8FEF8EBD0DB407FEFDCF8EB594
:101A30008FEF8EBD0DB407FEFDCF8EB581E090E037
:101A4000089580E090E008951F93CF93DF93EC0119
:101A5000162F0E94D30C8F3F19F080E090E031C028
:101A60001EBD0DB407FEFDCF1D3F19F481E090E0CF
:101A700028C090E088818EBD0DB407FEFDCF89811E
:101A80008EBD0DB407FEFDCF915011F02296F2CF1E
:101A90008FEF8EBD0DB407FEFDCF8FEF8EBD0DB461
:101AA00007FEFDCF8FEF8EBD0DB407FEFDCF8EB5C7
:101AB00090E08F71853009F091E081E09827892FBF
:101AC0009927DF91CF911F910895DF92EF92FF92B6
:101AD0000F931F93D82E7A018B010E94D30C8F3F56
:101AE00019F02FEF30E044C0DEBC0DB407FEFDCF8F
:101AF000812F9927AA27BB278EBD0DB407FEFDCFE6
:101B0000C801AA27BB278EBD0DB407FEFDCFBB279A
:101B1000A12F902F8F2D8EBD0DB407FEFDCFEEBCF3
:101B20000DB407FEFDCF80E4D81611F485E906C098
:101B300088E4D81611F487E801C080E08EBD0DB4AA
:101B400007FEFDCF8CE4D81631F48FEF8EBD0DB4B7
:101B500007FEFDCF8EB59AE08FEF8EBD0DB407FE68
:101B6000FDCF8EB5282F332787FF02C09150A1F7F4
:101B7000C9011F910F91FF90EF90DF900895882386
:101B800019F081E090E0089580910401992708956B
:101B900080910F01882319F0815080930F0180916B
:101BA0001001882319F081508093100190910E014B
:101BB00083B1817080930E01981749F480910401DC
:101BC00090FF02C0836001C08D7F8093040108955F
:101BD000A0E1B0E0EEEEFDE00C943811FA018823AC
:101BE00019F024E030E0DAC08A012A98633009F461
:101BF00082C0643028F4613079F0623051F474C0EE
:101C00006B3009F488C06C3009F49FC06A3009F465
:101C100078C024E030E0B8C040E050E060E070E020
:101C200089E40E94650D882309F0ACC060E170E092
:101C3000CE0101960E94EC0C882309F4A3C089818F
:101C400082958695869583707A8549858130C1F421
:101C5000872F99270196242F3327322F2227820F8F
:101C6000931FAA27BB276AE0880F991FAA1FBB1FD3
:101C70006A95D1F7F80180839183A283B38338C03A
:101C8000429546954695437028853327220F331F8A
:101C9000220F331F240F311D2F5F3F4F8F81992754
:101CA00083709070982F8827990F990F280F391FEC
:101CB000442755276E816F706E5F7370770F670FC3
:101CC0008B85881F8827881F860F9927099704C04E
:101CD000220F331F441F551F8A95D2F7F801208326
:101CE00031834283538304C080E092E091838083F8
:101CF00020E030E049C00E94D30C90E08F3F01F516
:101D00001EC08091040180FD47C040E050E060E0CB
:101D100070E089E409C08091040180FD3DC040E08D
:101D200050E060E070E08AE40E94650D882351F580
:101D300060E170E0C8010E94EC0C90E0811191E03C
:101D400081E09827292F33271FC08091040180FD4F
:101D500023C040E050E060E070E08AE70E94650D3B
:101D6000882381F490E08FEF8EBD0DB407FEFDCF88
:101D70008EB5F80180839F5F943009F4B9CF0F5F6F
:101D80001F4FF1CF21E030E02A9A8FEF8EBD0DB4C6
:101D900007FEFDCF8EB502C023E030E0C901E4E0CC
:101DA00060960C945411CF92DF92EF92FF920F93B2
:101DB000CF93DF93EB0169017A01882309F067C0B3
:101DC000002309F464C08091040180FF03C083E014
:101DD00090E05FC08091040182FF03C082E090E048
:101DE00058C080911101992782FD07C0E9E0CC0C11
:101DF000DD1CEE1CFF1CEA95D1F72A98013079F41E
:101E0000B701A60188E50E94650D882391F56EEF64
:101E1000CE010E94240D811181E008272AC081FF94
:101E20000EC040E050E060E070E087E70E94650D82
:101E3000402F55276627772787E50E94650DB70154
:101E4000A60189E50E94650D882399F46CEFCE0107
:101E50000E94240D882329F0015019F0C050DE4F54
:101E6000F5CF6DEF80E090E00E94240D882309F407
:101E700001E02A9A8FEF8EBD0DB407FEFDCF8EB51F
:101E800080E090E0002329F081E090E002C084E04F
:101E900090E0DF91CF910F91FF90EF90DF90CF9086
:101EA00008950F93CF93DF93EB01882309F050C07F
:101EB000002309F44DC08091040180FF03C083E03A
:101EC00090E048C08091110182FD07C0F9E0220F27
:101ED000331F441F551FFA95D1F72A98013081F41A
:101EE000BA01A90181E50E94650D882319F560E01A
:101EF00072E0CE010E94EC0C811181E008271AC02B
:101F0000BA01A90182E50E94650D882399F460E079
:101F100072E0CE010E94EC0C882329F0015019F0E8
:101F2000C050DE4FF4CF40E050E060E070E08CE461
:101F30000E94650D2A9A8FEF8EBD0DB407FEFDCF6E
:101F40008EB580E090E0002329F081E090E002C0AF
:101F500084E090E0DF91CF910F910895A4E0B0E08C
:101F6000E4EBFFE00C943611882319F081E090E057
:101F7000D0C08091040181FDC9C09AE08FEF8EBD71
:101F80000DB407FEFDCF8EB59150C1F72A9840E001
:101F900050E060E070E080E40E94650D813009F05F
:101FA000A0C084E680930F014AEA51E060E070E04F
:101FB00088E40E94650D813009F054C07E010894C8
:101FC000E11CF11C87019E012B5F3F4F8FEF8EBDFF
:101FD0000DB407FEFDCF8EB5F80181938F01E21796
:101FE000F307A1F78B81813009F07BC08C818A3A9D
:101FF00009F077C040E050E060E070E087E70E94C1
:10200000650D823048F440E050E060E070E489E61D
:102010000E94650D882321F080910F01882351F7DC
:1020200080910F01882309F45CC040E050E060E03B
:1020300070E08AE70E94650D882309F052C08FEF97
:102040008EBD0DB407FEFDCF8EB5F70181937F01E4
:10205000E017F107A1F7898186FF02C016E042C0B0
:1020600012E040C040E050E060E070E087E70E948E
:10207000650D823058F440E050E060E070E089E6A1
:102080000E94650D823010F412E001C011E01230A0
:1020900079F440E050E060E070E087E70E94650D71
:1020A000823078F440E050E060E070E089E605C0FE
:1020B00040E050E060E070E081E40E94650D88231C
:1020C00021F080910F01882311F780910F0188235F
:1020D00041F040E052E060E070E080E50E94650D74
:1020E000811110E0109311012A9A8FEF8EBD0DB46B
:1020F00007FEFDCF8EB5112321F0809104018E7F64
:1021000003C08091040181608093040180910401E7
:102110009927E6E024960C945211FB01DC0105900E
:102120000D920020E1F70895FB01DC0104C08D91C0
:102130000190801921F441505040C8F7881B990B39
:102140000895FB01DC0102C001900D924150504006
:10215000D8F70895DC0101C06D9341505040E0F77D
:102160000895FB01DC0101900D920020E1F7089534
:10217000FB019F01E8944230C4F04532B4F44A3088
:1021800029F497FB1EF4909581959F4F642F772734
:102190000E946111805D8A330CF0895D8193CB01CF
:1021A0000097A1F716F45DE251931082C9010C94D7
:1021B000D910DC01FC01672F71917723E1F7329789
:1021C00004C07C916D9370836291AE17BF07C8F312
:1021D0000895629FD001739FF001829FE00DF11D71
:1021E000649FE00DF11D929FF00D839FF00D749F91
:1021F000F00D659FF00D9927729FB00DE11DF91F3D
:10220000639FB00DE11DF91FBD01CF011124089599
:10221000A1E21A2EAA1BBB1BFD010DC0AA1FBB1FEA
:10222000EE1FFF1FA217B307E407F50720F0A21B5C
:10223000B30BE40BF50B661F771F881F991F1A94C9
:1022400069F760957095809590959B01AC01BD01F3
:10225000CF0108952F923F924F925F926F927F929B
:102260008F929F92AF92BF92CF92DF92EF92FF92A6
:102270000F931F93CF93DF93CDB7DEB7CA1BDB0B52
:102280000FB6F894DEBF0FBECDBF09942A883988F7
:1022900048885F846E847D848C849B84AA84B984FE
:1022A000C884DF80EE80FD800C811B81AA81B9810A
:1022B000CE0FD11D0FB6F894DEBF0FBECDBFED011E
:1022C0000895AA1BBB1B51E107C0AA1FBB1FA6177D
:1022D000B70710F0A61BB70B881F991F5A95A9F7CF
:0C22E00080959095BC01CD010895FFCFC2
:0622EC0046415400010010
:00000001FF
